:020000040000FA
:1000000055EF18F0120012000EEF00F01200010080
:1000100016310000600000006E000000DACFE4FF3F
:10002000E2CFDAFFE9CFE4FFEACFE4FFF6CFE4FF67
:10003000F7CFE4FFF5CFE4FFF3CFE4FFF4CFE4FF25
:10004000FACFE4FF00EE00F0140EE80403E3EECF75
:10005000E4FFFBD700EE14F0080EE80403E3EECF54
:10006000E4FFFBD7E6529D50200B30E09E50200B62
:100070002DE0E1EC17F001014F6FABA407D0AB9E70
:10008000A2814D2B000E4E23AB8E01D0A291ABA2CC
:1000900007D0AB98A283AB884B2B000E4C2301D02A
:1000A000A293ACA2FED7010149C1E9FF4AC1EAFF10
:1000B000492B000E4A234FC1EFFFF90E495D010E97
:1000C0004A5904E3A90E496F010E4A6FE55200EE4A
:1000D0001BF0080EE80403E3E5CFEDFFFBD700EECD
:1000E00013F0140EE80403E3E5CFEDFFFBD7E5CFF3
:1000F000FAFFE5CFF4FFE5CFF3FFE5CFF5FFE5CF5E
:10010000F7FFE5CFF6FFE5CFEAFFE5CFE9FFE5CF63
:10011000DAFF1100D9CFE6FFE1CFD9FF040EE126C7
:100120008B908B928B960000000000000000800EE8
:10013000F36E020EF3CFDBFF030EDB6ADE6ADD6ACD
:10014000DECF14F0DDCF15F0D890155004E6080E80
:10015000145C000E155835E2FE0EDB50166E176A61
:10016000020EDB501614146E030EDB501714156EBE
:10017000020EDB50141803E1030EDB50151802E1E8
:100180008B8201D08B9200000000000000008B8663
:100190000000000000000000020EDBCF14F0030E90
:1001A000DBCF15F0D89015321432020E14C0DBFFED
:1001B000030E15C0DBFF8B96DF2A010E01E3DB2A5D
:1001C000BFD7800EF36E020EF3CFDBFF030EDB6AA8
:1001D000DE6ADD6ADECF14F0DDCF15F0D890155061
:1001E00004E6080E145C000E155835E2FD0EDB50D7
:1001F000166E176A020EDB501614146E030EDB50D7
:100200001714156E020EDB50141803E1030EDB50B9
:10021000151802E18B8201D08B92000000000000D3
:1002200000008B860000000000000000020EDBCF03
:1002300014F0030EDBCF15F0D89015321432020EF5
:1002400014C0DBFF030E15C0DBFF8B96DF2A010E07
:1002500001E3DB2ABFD700008B80040EE15C02E2E1
:10026000E16AE552E16EE552E7CFD9FF1200D9CF3E
:10027000E6FFE1CFD9FF00D0E552E7CFD9FF12006A
:10028000700ED36E330EE66EE66A740EE66E18ECF0
:1002900017F0E552E552E5529F8AD08E9D9AF29C66
:1002A000F29E1200D9CFE6FFE1CFD9FF020EE12680
:1002B000DE6ADD6AFD0EDBCFE9FFFE0EDBCFEAFF73
:1002C000EF5016E0FD0EDBCFE9FFFE0EDBCFEAFFBD
:1002D000EF50E66EE66A1FD8E552E552DF2A010EBE
:1002E00001E3DB2AFD0EDB2AFE0E01E3DB2AE2D767
:1002F000DECF14F0DDCF15F014C0F3FF15C0F4FF0E
:10030000020EE15C03E200D0E16AE552E16EE552E3
:10031000E7CFD9FF1200D9CFE6FFE1CFD9FFACA2DA
:10032000FED7FD0EDBCFE6FF1CEC18F0E552E552E0
:10033000E7CFD9FF12000D0EE66EE66AECDFE5525C
:10034000E5520A0EE66EE66AE6DFE552E552120075
:10035000D9CFE6FFE1CFD9FF0A0EE1260101BC0E9D
:10036000446F000E456FFC0EDBCF14F0010EE76EFC
:100370001418E8AE02D0143403D0E750D8801454D7
:1003800001E2DBD0FC0EDB5028E1FD0EDBCF14F0E8
:10039000FE0EDBCF15F0060E14C0DBFF070E15C0F6
:1003A000DBFF080EDB6A090EDB6A44C1E6FF45C1CC
:1003B000E6FFD950060FE96EDACFEAFFEECFE6FF8F
:1003C000EECFE6FFEECFE6FFEFCFE6FF8DEC14F0C9
:1003D000146E060EE15E145010D044C1E6FF45C114
:1003E000E6FFFD0EDBCFE6FFFE0EDBCFE6FFF3EC14
:1003F00013F0E552E552E552E5520101A1AD84D07A
:10040000BC0EE66E000EE66E5FEC16F0E552E552AD
:10041000020EF3CFDBFF030EF4CFDBFFDE6ADD6AF3
:10042000DECF14F0DDCF15F0020EDBCF16F0030E99
:10043000DBCF17F01650145C175015582EE2020E41
:10044000DBCF16F0030EDBCF17F0DE50165CE96E43
:10045000DD501758EA6EE906000EEA5ABC0EE9268E
:10046000000EEA22EF50E66EFC0EDB50040F146E15
:10047000156A14BE1568DE50145CE96EDD5015581F
:10048000EA6EBC0EE926000EEA22E552E750EF6E56
:10049000DF2A010E01E3DB2AC3D7DE6ADD6ADECF85
:1004A00014F0DDCF15F0FC0EDB50050F186E196A45
:1004B00018BE1968020EDB50185C166E030EDB5076
:1004C0001958176E1650145C175015581DE201018B
:1004D000A1A90BD0DECFE9FFDDCFEAFFBC0EE926F4
:1004E000000EEA22300EEF6E0AD0DECFE9FFDDCF3C
:1004F000EAFFBC0EE926000EEA22200EEF6EDF2A8C
:10050000010E01E3DB2ACBD7FC0EDB50050FE96EB1
:10051000EA6AE9BEEA68BC0EE926000EEA22EF6A42
:1005200044C1E6FF45C1E6FFBDDEE552E552020EDD
:10053000F3CFDBFF030EF4CFDBFF0A0EE15C02E238
:10054000E16AE552E16EE552E7CFD9FF1200D9CF5B
:10055000E6FFE1CFD9FF0E0EE126F90EDBCFDEFF7D
:10056000DBCFDDFFF80EDBCF16F0000EE76E1618BE
:10057000E8AE02D0163403D0E750D880165402E318
:10058000070E12D0F80EDBCF17F0160EE76E171815
:10059000E8AE02D0173403D0E750D880175402E2F7
:1005A000170E02D0F80EDB28146E156A14BE1568FB
:1005B000080E14C0DBFF090E15C0DBFF020EDB6A5C
:1005C000030EDB6AFB0EDBCF14F0FC0EDBCF15F065
:1005D000FD0EDBCF16F0FE0EDBCF17F00A6A0B6ABA
:1005E0000C6A0D6A14C005F015C006F016C007F0BD
:1005F00017C008F0E2EC12F0010A33E1F90EDBCF8C
:10060000E9FFDB2AFA0EDBCFEAFF01E3DB2A2D0E3E
:10061000EF6EFB0EDBCF14F0FC0EDBCF15F0FD0E02
:10062000DBCF16F0FE0EDBCF17F00A6A0B6A800EE6
:100630000C6EBF0E0D6E14C005F015C006F016C08E
:1006400007F017C008F03DEC12F0FB0E05C0DBFF11
:10065000FC0E06C0DBFFFD0E07C0DBFFFE0E08C070
:10066000DBFFFB0EDBCF14F0FC0EDBCF15F0FD0E35
:10067000DBCF16F0FE0EDBCF17F00A6A0B6A0C6AAE
:100680000D6A14C005F015C006F016C007F017C0BB
:1006900008F0D9EC12F0010A4AE1FB0EDBCF14F0AE
:1006A000FC0EDBCF15F0FD0EDBCF16F0FE0EDBCF20
:1006B00017F00A6A0B6A800E0C6E3F0E0D6E14C0A6
:1006C00005F015C006F016C007F017C008F0E2EC00
:1006D00012F0010A2CE1146A156A200E166E410E02
:1006E000176ED950FB0FE96EFF0EDA20EA6EEECFDF
:1006F00005F0EECF06F0EECF07F0EFCF08F014C014
:100700000AF015C00BF016C00CF017C00DF03DEC50
:1007100012F008C0EDFF07C0EDFF06C0EDFF05C0F9
:10072000EFFF020EDB06030E01E2DB06B6D7FB0E7F
:10073000DBCF14F0FC0EDBCF15F0FD0EDBCF16F097
:10074000FE0EDBCF17F00A6A0B6A200E0C6E410E0C
:100750000D6E14C005F015C006F016C007F017C0E6
:1007600008F0E2EC12F0010A2EE0FB0EDBCF14F0F1
:10077000FC0EDBCF15F0FD0EDBCF16F0FE0EDBCF4F
:1007800017F00A6A0B6A200E0C6E410E0D6E14C033
:1007900005F015C006F016C007F017C008F0EAEC27
:1007A00011F0FB0E05C0DBFFFC0E06C0DBFFFD0EEB
:1007B00007C0DBFFFE0E08C0DBFF020EDB2A030EC4
:1007C00001E3DB2AB4D7020EDBCF14F0030EDBCF3C
:1007D00015F0D950080FE96EDACFEAFF1450EE2673
:1007E0001550ED22010EF36E040EF3CFDBFF050E64
:1007F000DB6A040EDBCF06F0050EDBCF07F040EC22
:1008000011F00A0E05C0DBFF0B0E06C0DBFF0C0E5D
:1008100007C0DBFF0D0E08C0DBFF040EDBCF14F0BA
:10082000050EDBCF15F0080EDBCF16F0090EDBCF7F
:1008300017F015501718E8AE02D0173404D0165030
:10084000145C175015582EE20A0EDBCF14F00B0E75
:10085000DBCF15F00C0EDBCF16F00D0EDBCF17F053
:100860000A6A0B6A200E0C6E410E0D6E14C005F064
:1008700015C006F016C007F017C008F0EAEC11F03A
:100880000A0E05C0DBFF0B0E06C0DBFF0C0E07C017
:10089000DBFF0D0E08C0DBFF040EDB2A050E01E3B3
:1008A000DB2ABBD70A0EDBCF18F00B0EDBCF19F01B
:1008B0000C0EDBCF1AF00D0EDBCF1BF00A6A0B6AB1
:1008C0000C6A400E0D6E18C005F019C006F01AC073
:1008D00007F01BC008F0EAEC11F005C014F006C0E8
:1008E00015F007C016F008C017F0D950FB0FE96EDD
:1008F000FF0EDA20EA6EEECF05F0EECF06F0EECF77
:1009000007F0EFCF08F014C00AF015C00BF016C0C6
:100910000CF017C00DF054EC11F008C0EDFF07C04B
:10092000EDFF06C0EDFF05C0EFFFFB0EDBCF14F0BF
:10093000FC0EDBCF15F0FD0EDBCF16F0FE0EDBCF8D
:1009400017F00A6A0B6A200E0C6E410E0D6E14C071
:1009500005F015C006F016C007F017C008F0E2EC6D
:1009600012F0010A13E0FB0EDB6AFC0EDB6A800E5C
:10097000F36EFD0EF3CFDBFF3F0EF36EFE0EF3CFF3
:10098000DBFF020EDB2A030E01E3DB2A020EDBCFC4
:1009900014F0030EDBCF15F00001800E15145FE09C
:1009A000F90EDBCFE9FFDB2AFA0EDBCFEAFF01E32A
:1009B000DB2A300EEF6EF90EDBCFE9FFDB2AFA0EF1
:1009C000DBCFEAFF01E3DB2A2E0EEF6E080EDBCF52
:1009D00014F0090EDBCF15F0800E151414E0020E92
:1009E000DBCF16F0030EDBCF17F0080EDB50165CE2
:1009F000146E090EDB501758156E020E14C0DBFF83
:100A0000030E15C0DBFF040EDB68050EDB68040E69
:100A1000DBCF14F0050EDBCF15F0020EDBCF16F0A6
:100A2000030EDBCF17F017501518E8AE02D01534BF
:100A300004D01450165C1550175811E2F90EDBCF94
:100A4000E9FFDB2AFA0EDBCFEAFF01E3DB2A300EF7
:100A5000EF6E040EDB06050E01E2DB06D8D7040EAE
:100A6000DB6A050EDB6A040EDBCF14F0050EDBCF6C
:100A700015F0080EDBCF16F0090EDBCF17F015507E
:100A80001718E8AE02D0173404D01650145C175073
:100A9000155801E3ACD0FB0EDBCF05F0FC0EDBCF2D
:100AA00006F0FD0EDBCF07F0FE0EDBCF08F0AAEC60
:100AB00012F0060E06C0DBFF070E07C0DBFF300E8C
:100AC000E76E060EDBCF14F0070EDBCF15F0E75014
:100AD0001426000E1522F90EDBCFE9FFDB2AFA0EF1
:100AE000DBCFEAFF01E3DB2A14C0EFFF040EDBCF0C
:100AF00014F0050EDBCF15F0020EDB50141803E1E5
:100B0000030EDB5015180BE1F90EDBCFE9FFDB2AF2
:100B1000FA0EDBCFEAFF01E3DB2A2E0EEF6E060EA4
:100B2000DBCF06F0070EDBCF07F040EC11F00A0E2A
:100B300005C0DBFF0B0E06C0DBFF0C0E07C0DBFFA2
:100B40000D0E08C0DBFF05C014F006C015F007C08D
:100B500016F008C017F0D950FB0FE96EFF0EDA202F
:100B6000EA6EEECF05F0EECF06F0EECF07F0EFCF56
:100B700008F014C00AF015C00BF016C00CF017C036
:100B80000DF053EC11F008C0EDFF07C0EDFF06C0FB
:100B9000EDFF05C0EFFF146A156A200E166E410EB8
:100BA000176ED950FB0FE96EFF0EDA20EA6EEECF1A
:100BB00005F0EECF06F0EECF07F0EFCF08F014C04F
:100BC0000AF015C00BF016C00CF017C00DF03DEC8C
:100BD00012F008C0EDFF07C0EDFF06C0EDFF05C035
:100BE000EFFF040EDB2A050E01E3DB2A3CD7F90EEA
:100BF000DBCFE9FFFA0EDBCFEAFFEF6ADECF14F0BE
:100C0000DDCF15F014C0F3FF15C0F4FF0E0EE15C4C
:100C100003E200D0E16AE552E16EE552E7CFD9FF89
:100C20001200D9CFE6FFE1CFD9FFE652800EDF6E8A
:100C3000DF50000817E2FE0EDB50DF1408E0310E33
:100C4000E66EE66A8BEC01F0E552E55207D0300E15
:100C5000E66EE66A8BEC01F0E552E552DF407F0B71
:100C6000DF6EE6D7E552E552E7CFD9FF1200D9CFC4
:100C7000E6FFE1CFD9FF020EE126FE0EDB50F00BBE
:100C8000E8380F0B300FDF6EDF50390803E2070E34
:100C9000DF24DF6EFE0EDB500F0B300FE76E010E10
:100CA000E7CFDBFFDB5039080AE2070E146E010EB6
:100CB000DBCFE7FF1450E726010EE7CFDBFFDFCFE6
:100CC000E6FFE66A8BEC01F0E552E552010EDBCF60
:100CD000E6FFE66A8BEC01F0E552E552680EE66E3F
:100CE000E66A8BEC01F0E552E552020EE15C02E2AD
:100CF000E16AE552E16EE552E7CFD9FF1200D9CFA4
:100D0000E6FFE1CFD9FF020EE126DE6ADD6ADECF23
:100D100014F0DDCF15F0FE0EDB50000115AE02D051
:100D2000D89003D0145C000E15580CE2200EE66E2D
:100D3000E66A8BEC01F0E552E552DF2A010E01E391
:100D4000DB2AE5D7020EE15C02E2E16AE552E16EE0
:100D5000E552E7CFD9FF1200D9CFE6FFE1CFD9FFA7
:100D6000FF0EE76EFD0EDBCF14F0FE0EDBCF15F0AD
:100D7000E7501416156A1450A96EFD0EDBCF14F05F
:100D8000FE0EDBCF15F015C014F0156A030E141417
:100D9000AA6EA69EA69CA680A85000D0E552E7CFDA
:100DA000D9FF1200D9CFE6FFE1CFD9FF020EE1262D
:100DB000DE6ADD6AFF0EE76EFD0EDBCF14F0FE0E7D
:100DC000DBCF15F0E7501416156A1450A96EFD0E0E
:100DD000DBCF14F0FE0EDBCF15F015C014F0156A52
:100DE000030E1414AA6EFC0EDB50A86EA69EA684F9
:100DF000A69CF2AE04D0F29E010EDE6EDD6A550EA8
:100E0000A76EAA0EA76EA682A1A8FED7A198A69447
:100E1000D9CFE9FFDACFEAFF010EEE1801E1ED507C
:100E200001E1F28E020EE15C02E2E16AE552E16E5E
:100E3000E552E7CFD9FF1200D9CFE6FFE1CFD9FFC6
:100E4000FB0EDBCFE9FFFC0EDBCFEAFFEF501DE02E
:100E5000FB0EDBCFE9FFDB2AFC0EDBCFEAFF01E371
:100E6000DB2AEF50E66EFD0EDBCF14F0DB2AFE0E20
:100E7000DBCF15F001E3DB2A14C0E6FF15C0E6FF67
:100E800091DFE552E552E552DBD7E552E7CFD9FFD6
:100E90001200D9CFE6FFE1CFD9FFE652D950FD0FBE
:100EA000E96EFF0EDA20EA6EFF0ED880EE54030ED4
:100EB000ED5401E21BD0FD0EDBCFE6FFFE0EDBCFD3
:100EC000E6FF4ADFE552E552DF6EDF5001E10ED06A
:100ED000DFCFE6FFE66A8BEC01F0E552E552FD0E4E
:100EE000DB2AFE0E01E3DB2ADF50D8E1E80EE66ED6
:100EF000030EE66EE66AE66A37EC01F0E552E5526B
:100F0000E552E552E552E552E7CFD9FF12000F0155
:100F1000396B8168936893809382939493869388C6
:100F2000938A938C938E386B3881388338850F0E73
:100F3000926E3A6B8268840E946E9490949294842C
:100F400094969498949A949C948E606A8B6A1200FA
:100F5000040EE66E010EE66E5FEC16F0E552E55209
:100F6000F3CF5EF1F4CF5FF10101080E5E5D000E7C
:100F70005F591DE2A90E146E2D0E156E166A14C06F
:100F8000E6FF15C0E6FF16C0E6FFFE0EE66EE66859
:100F9000F8EC15F0176E050EE15E1750F3CF60F117
:100FA000F4CF61F101015E2B000E5F23DDD7090E46
:100FB000E66EE66A040EE66E010EE66EA40E146E90
:100FC0002D0E156E166A14C0E6FF15C0E6FF16C09A
:100FD000E6FFFE0EE66EE668F8EC15F0176E090EF9
:100FE000E15E1750F3CF60F1F4CF61F11200C280DF
:100FF000C19EC08EC08AC088C096C082C094C09076
:10100000C196C194C192C1901200D9CFE6FFE1CF41
:10101000D9FF020EE126FD0EDBCF14F0FE0EDBCF72
:1010200015F0D89014361536D89014361536010EB2
:101030001424C26E010EE66EE66A6EEC15F0E552FF
:10104000E55288EC18F083EC18F0000901E0FBD7BA
:1010500071EC18F0F3CFDEFFF4CFDDFFDECF14F03C
:10106000DDCF15F014C0F3FF15C0F4FF020EE15CF4
:1010700003E200D0E16AE552E16EE552E7CFD9FF25
:101080001200CD9ECD9CCD8ACD88CD96CD94CD82BB
:10109000CD90CC9ECC9ACC92CC909F80D08EDB0E03
:1010A000E66E0B0EE66E00EC18F0E552E5529E90EF
:1010B000F29CCD909D90F29EF29C1200600ED36E39
:1010C0009B6A9B9C24DF8B8089980101466BBC0E38
:1010D000446F000E456F6C0E026F000E036F716B54
:1010E000726B6F6B706B736B746B0101A96B010199
:1010F000A90E496F010E4A6F49C147F14AC148F133
:10110000A26BA28DA289A295A29BA297A291A29363
:101110004D6B4E6B4B6B4C6B40EC01F00101A19F92
:1011200089880C0EE66EE66A8BEC01F0E552E5521A
:10113000F40EE66E010EE66E6EEC15F0E552E55229
:101140000101506B516B006B016B9BEC01F00101D5
:101150006C0E026F000E036F02C1E6FF03C1E6FFD3
:1011600052EC01F0E552E552F3CF60F1F4CF61F1BA
:101170009BEC01F001016C0E026F000E036F62C068
:1011800014F063C015F0166A14C0E6FF15C0E6FF40
:1011900016C0E6FF02C1E6FF03C1E6FF46EC16F00B
:1011A000176E050EE15E175002C1E6FF03C1E6FFB0
:1011B00052EC01F0E552E552F3CF60F1F4CF61F16A
:1011C000E80EE66E030EE66EE66AE66A37EC01F0BC
:1011D000E552E552E552E55266C014F067C015F0DD
:1011E000166A14C0E6FF15C0E6FF16C0E6FF02C18E
:1011F000E6FF03C1E6FF46EC16F0176E050EE15E52
:10120000175002C1E6FF03C1E6FF52EC01F0E552C0
:10121000E552F3CF60F1F4CF61F1E80EE66E030E14
:10122000E66EE66AE66A37EC01F0E552E552E55211
:10123000E552000EE66EE66A2CDEE552E552200E1F
:10124000E66EE66A26DEE552E552600EE66EE66A76
:1012500020DEE552E552A00EE66EE66A1ADEE552A1
:10126000E552C00EE66EE66A14DEE552E5529BECEE
:1012700001F0100EE66E270EE66EE66AE66A37ECBF
:1012800001F0E552E552E552E5528B6AB0DEE66ABE
:10129000400EE66E8AEC00F0E552E552E66A410E39
:1012A000E66E8AEC00F0E552E5520101956B966B13
:1012B000A00E976F400E986F090EE66EE66A040E58
:1012C000E66E040EE66E010EE66E95C1E6FF96C16F
:1012D000E6FF97C1E6FF98C1E6FFA7EC02F0166EA5
:1012E000070EE15E1650F3CF14F0F4CF15F014C0E2
:1012F000E6FF15C0E6FF870E176E2D0E186E196AF1
:1013000017C0E6FF18C0E6FF19C0E6FFFE0EE66E46
:10131000E668F8EC15F01A6E090EE15E1A50F3CF8C
:1013200060F1F4CF61F19BEC01F001015E6B5F6B4A
:10133000686B696B050EE66E400EE66E8AEC00F097
:10134000E552E552E66A410EE66E8AEC00F0E5529F
:10135000E552C80EE66EE66A6EEC15F0E552E5520F
:10136000000EE66EE66A51DEE552E552F3CF6AF111
:10137000F4CF6BF1010168516A25686F69516B21E7
:10138000696F6AC106F06BC107F03EEC11F005C051
:1013900014F006C015F007C016F008C017F00A6A6E
:1013A0000B6A480E0C6E3D0E0D6E14C005F015C094
:1013B00006F016C007F017C008F03DEC12F005C0AB
:1013C00095F106C096F107C097F108C098F1090E93
:1013D000E66EE66A020EE66E040EE66E010EE66E3C
:1013E00095C1E6FF96C1E6FF97C1E6FF98C1E6FF0B
:1013F000A7EC02F0166E070EE15E1650F3CF14F064
:10140000F4CF15F014C0E6FF15C0E6FF6AC1E6FF91
:101410006BC1E6FF590E176E2D0E186E196A17C0B4
:10142000E6FF18C0E6FF19C0E6FFFE0EE66EE668AE
:10143000F8EC15F01A6E0B0EE15E1A50F3CF60F166
:10144000F4CF61F1E66A400EE66E8AEC00F0E552F8
:10145000E552010EE66E410EE66E8AEC00F0E552B2
:10146000E552C80EE66EE66A6EEC15F0E552E552FE
:10147000000EE66EE66AC9DDE552E552F3CF6AF189
:10148000F4CF6BF16AC106F06BC107F03EEC11F0CE
:1014900005C018F006C019F007C01AF008C01BF00C
:1014A0000A6A0B6AA00E0C6E400E0D6E18C005F095
:1014B00019C006F01AC007F01BC008F03DEC12F08E
:1014C00005C014F006C015F007C016F008C017F0EC
:1014D0000A6A0B6A800E0C6E440E0D6E14C005F085
:1014E00015C006F016C007F017C008F0EAEC11F0BE
:1014F00005C095F106C096F107C097F108C098F1B4
:10150000090EE66EE66A020EE66E040EE66E010E47
:10151000E66E95C1E6FF96C1E6FF97C1E6FF98C16A
:10152000E6FFA7EC02F0166E070EE15E1650F3CF51
:1015300014F0F4CF15F014C0E6FF15C0E6FF6AC141
:10154000E6FF6BC1E6FF3B0E176E2D0E186E196A93
:1015500017C0E6FF18C0E6FF19C0E6FFFE0EE66EF4
:10156000E668F8EC15F01A6E0B0EE15E1A50F3CF38
:1015700060F1F4CF61F101015E2B000E5F230F0ECD
:10158000D8805E55000E5F5564E268C106F069C1FF
:1015900007F03EEC11F005C014F006C015F007C0CE
:1015A00016F008C017F0070E0A6E0B6A480E0C6E94
:1015B0003B0E0D6E14C005F015C006F016C007F006
:1015C00017C008F03DEC12F005C095F106C096F189
:1015D00007C097F108C098F1020EE66E040EE66EA1
:1015E000010EE66E95C1E6FF96C1E6FF97C1E6FFE4
:1015F00098C1E6FFA7EC02F0166E070EE15E1650EA
:10160000F3CF14F0F4CF15F014C0E6FF15C0E6FFD9
:1016100068C1E6FF69C1E6FF240E176E2D0E186E35
:10162000196A17C0E6FF18C0E6FF19C0E6FFFE0EF4
:10163000E66EE668F8EC15F01A6E090EE15E1A50D7
:10164000F3CF60F1F4CF61F101015E6B5F6B686B0A
:10165000696B9BEC01F06ED6120069EC10F0FB0E8A
:10166000DBCFF3FFDB06F35000090AE0B7EC10F024
:10167000FA0E22EC11F0F3E1151CF1E1010E01D09C
:10168000000E98EF10F069EC10F03B0EE12402E33D
:10169000E168E652E16E010EDB6A020EDB6AF90ECA
:1016A000DBCFF6FFFA0EDBCFF7FFFB0EDBCFF8FF49
:1016B0000800F550DF6EDF5002E1BCEF0FF0250EA1
:1016C000DF5C02E0AFEF0FF0030EDB6A040EDB6AB3
:1016D000050EDB6A060EDB6A070EDB6AD1EC0FF043
:1016E0002D0EDF5C0CE02B0EDF5C09E0200EDF5CD2
:1016F00006E0230EDF5C03E0300EDF5C1AE1DF5012
:10170000300A14E0130A0FE0030A0AE00B0A05E0AE
:10171000060AE4E1030EDB80E1D7030EDB82DED7AD
:10172000030EDB84DBD7030EDB86D8D7030EDB8802
:10173000D5D72A0EDF5C1BE1CDEC0FF01BEC10F0CF
:1017400010E0030EDB8006680768130EDBCF0BF09A
:10175000140EDBCF0CF0C6EC13F0040E04C0DBFF5C
:1017600003D0130E04EC10F0D1EC0FF00BD0090EE7
:10177000DB6A72EC10F003E0E6EC10F0FAD7090E29
:1017800004EC10F0030EDBB0DB982E0EDF5C1BE1E7
:10179000D1EC0FF02A0EDF5C0BE1CDEC0FF01BEC6F
:1017A00010F003E1130E56EC10F0D1EC0FF00BD05B
:1017B000090EDB6A72EC10F003E0E6EC10F0FAD7E9
:1017C000090E56EC10F0680EDF5C07E1D1EC0FF06B
:1017D000680EDF5C1DE1030E18D0740EDF5C17E0AD
:1017E0007A0EDF5C14E0480EDF5C06E0540EDF5C2E
:1017F00003E05A0EDF5C02E1020E07D06C0EDF5CE4
:1018000003E06A0EDF5C04E1010EA9EC10F0C9DB15
:10181000DF506E0A01E17FD31E0A01E192D1200A56
:1018200001E18FD13F0A01E149D11A0A01E146D114
:101830000D0A01E143D1200A01E140D13A0A01E158
:101840003DD1200A01E13AD1260A01E135D10D0A44
:1018500001E132D11A0A01E1D9D0200A4AE0300A66
:101860001FE0460A0EE0250A01E083D3D950F90FA4
:10187000E96EFF0EDA20EA6E010EEE5E000EEE5A01
:10188000EE5AB7EC10F0250EE66E95DB03E1151C61
:1018900001E169D3B3EC10F001E26BD3DB2A69D329
:1018A000080EDB6A040EDB50010806E2040EDB04BE
:1018B0007BEC10F0DB508BDB080EDB5009E0030EF5
:1018C000DB50010B05E172DB01E04DD3080EDB6A52
:1018D00064DBEFCFDFFF2BEC11F003E1151C01E11E
:1018E00042D3B3EC10F001E3DB2A60DB01E141D32A
:1018F0003AD3070EDB5002080FE1F7EC10F0030EAD
:10190000BEEC10F00E0EEECFDBFF0F0EEECFDBFFC6
:10191000100EEECFDBFF20D0F70EDBCF17F0F80E66
:10192000DBCF18F0020E175E000E185AF70E17C024
:10193000DBFFF80E18C0DBFF17C0E9FF18C0EAFF95
:10194000AEEC10F0166A0E0E14C0DBFF0F0E15C0C1
:10195000DBFF100E16C0DBFF0E0EDBCFE6FF0F0E17
:10196000DBCFE6FF100EDBCFE6FF6DEC16F0E552A5
:10197000E552E552130E05C0DBFF140E06C0DBFF77
:10198000060EDB5005E0130EF2EC10F001E26ADB0C
:1019900016EC11F002E2130E37DBD9EC10F006E082
:1019A000040EF2EC10F002E2050E2EDB030EDBB0AB
:1019B00005D0FCDA01E0D7D2080EDB6A090EDB6A3B
:1019C0000E0EDBCFF6FF0F0EDBCFF7FF100EDBCFD7
:1019D000F8FF0800F550DF6EDF5014E01CEC11F04A
:1019E00011E22BEC11F003E1151C01E1BCD2BBDBD1
:1019F00001E3DB2A090EDB2AD9500E0FE96E000E37
:101A0000CBDBE7D7D3DA01E1B4D2ADD2C6DA110E1F
:101A1000EECFDBFF120EEDCFDBFF110EDBCFE6FFCB
:101A2000120EDBCFE6FF5FEC16F0E552E552130E27
:101A3000F3CFDBFF140EF4CFDBFF060EDB5004E028
:101A4000130ED0DB01E20EDB16EC11F002E2130EF6
:101A5000DBDAAFDB05E0040EC5DB02E2050ED4DA0B
:101A6000030EDBB005D0A2DA01E07DD2080EDB6AFE
:101A7000090EDB6A110EDBCFE9FF120EDBCFEAFFA6
:101A8000EFCFDFFFDF5014E0D7DB12E2E4DB03E14E
:101A9000151C01E168D267DB01E3DB2A090EDB2AB2
:101AA000110EDB2ADBCFE9FF120EE8E3DB2AE6D7D3
:101AB0007DDA01E15ED257D2030EDB8E070EDB0426
:101AC00010E195DB040E5ADB0A0EEECFDBFF0B0EA6
:101AD000EECFDBFF0C0EEECFDBFF0D0EEECFDBFF0C
:101AE0006CD0070EDB5003082CE1030EDBAE0DD0EB
:101AF000B2DA020E76DAEFCF14F0156A166A176AB8
:101B000014AE39D01568166835D0F70EDBCF15F056
:101B1000F80EDBCF16F0020E155E000E165AF70E09
:101B200015C0DBFFF80E16C0DBFF15C0E9FF16C0BD
:101B3000EAFFEFCF14F00A0E14C0DBFF0B0EDB6AD6
:101B400038D0070EDB50020809E1030EDBAE04D0EB
:101B500059DB16AE10D00ED055DB0DD0030EDBAE28
:101B600012D079DA020E3DDAF9DA166A176A15AE82
:101B700002D016681768E2DA0C0E16C0DBFF0D0EF5
:101B800017C0DBFF1AD0F70EDBCF16F0F80EDBCF55
:101B900017F0020E165E000E175AF70E16C0DBFF86
:101BA000F80E17C0DBFF16C0E9FF17C0EAFFD6DA50
:101BB000C5DA0C0EDB6A0D0EDB6A060EDB5005E1A2
:101BC000010EF36E050EF3CFDBFF150EDB6A160E6A
:101BD000DB6AD950370F146E000EDA20156E390EFD
:101BE00014C0DBFF3A0E15C0DBFF380EDB6A080EAF
:101BF000DB6A0A0EAEDADF50780A12E0200A10E043
:101C0000280A0CE0200A0AE03F0A06E00D0A02E07A
:101C1000200A08E1020E05D0080E03D0080EDF26C8
:101C2000100E97DA030EDBBE02D0DB92DB94DB50A2
:101C3000800B24E08ADAD890030EEB50000A08E605
:101C4000000EEE5C000EEE58000EEE58000EEE5840
:101C500015E213DA09680A680B680C6851EC17F092
:101C60000A0E00C0DBFF0B0E01C0DBFF0C0E02C032
:101C7000DBFF0D0E03C0DBFF2D0E08D0030EDBA231
:101C800002D02B0E03D0DBA408D0200EF36E170E6B
:101C9000F3CFDBFF150EDB2A02D0170EDB6A050E31
:101CA000DB5003E1B7D901E189D0F40E146E300E98
:101CB000156E000E166E070EDBCF17F0186A196A44
:101CC0001A6A17C009F018C00AF019C00BF01AC040
:101CD0000CF0D3D9BDEC17F014500024F36E15505E
:101CE0000120F46E16500220F86EF4CFF7FFF3CF08
:101CF000F6FF0800090EF5CFDBFF580EDF5C0FE1A1
:101D0000610EF36E090E7BD90AE3200E146E090EE4
:101D1000DBCFE7FF1450E75E090EE7CFDBFF070ECE
:101D2000DBCF14F0156A166A176A0FDA14C009F0CF
:101D300015C00AF016C00BF017C00CF0EECF04F07F
:101D4000EECF05F0EECF06F0EFCF07F0BDEC17F0C9
:101D500007C0EDFF06C0EDFF05C0EDFF04C0EFFFBB
:101D6000390EDBCFE9FFDB063A0EDBCFEAFF01E2FB
:101D7000DB06090EDBCFEFFF150EDB2A4BD995E111
:101D8000030EDBA61DD06F0EDF5C06E1C1D918E3A0
:101D9000150EDB285BDA14D0780EDF5C09E0580EF4
:101DA000DF5C06E0620EDF5C03E0420EDF5C08E110
:101DB000020EF36E160EF3CFDBFF02D0150EDB6AB8
:101DC000030EDB50100B0EE0040EDBCF14F0050EFB
:101DD000DB50D880145406E2060EDB5003E1040EFB
:101DE000DB5034DA95D90AE2050EDBCFE7FF150E9A
:101DF000DB50E75E050EE7CFDBFF02D0050EDB6AA6
:101E0000040EDBCF14F0160E45D9D880145414E21A
:101E1000160EDBCFE6FF150EDBCFE6FF040EDBCFA1
:101E2000E6FF050EDB50E552E75CE552D880E7544B
:101E3000E552D880E7545FD9030EDB50010B0BE16C
:101E4000080EDB5008E0B2D801E08DD0080EDB5060
:101E5000BED8080EDB6A170EDB5007E088D9170ED4
:101E6000F1D903E1151C01E17ED0160EDB5016E01E
:101E70007ED9300EE66E9FD802E1151C74E077D94A
:101E8000DFCFE6FFD6EC16F0E552E552E552F4CF8F
:101E900015F00001F31C02E1151C65E0050EDBCF17
:101EA00014F0160EDB50D880145409E2050EDBCF77
:101EB000E7FF160EDB50E75E050EE7CFDBFF300EC7
:101EC000E66E050ECBD94FE1390EDB2ADBCFE9FFF9
:101ED0003A0E01E3DB2ADBCFEAFF090EEFCFDBFF8F
:101EE000DB500EE044D9090EADD902E1151C3BE0F0
:101EF000390EDB2ADBCFE9FF3A0EEDE3DB2AEBD725
:101F000055D831E1160EDBCFE6FF080EC3D8E552F7
:101F1000E7245DD82ED0070EDB50030A1CE0010A2F
:101F200014E0030A07E07BD9DBCFEEFF020EDBCF24
:101F3000EDFF1FD0F5D8196A17AE02D018681968DE
:101F40002CD8BCD819C0EEFF14D0EAD817BE186838
:101F500024D8B4D80ED063D9DBCFEFFF0AD07BD919
:101F600005E1151C03E1F368F46810D0FCD801E327
:101F7000DB2A79D958EF0BF0010EDBCF14F0020EFB
:101F8000DBCF15F014C0F3FF15C0F4FF3B0EE15C8E
:101F900002E2E16AE552E16ECBD029D9020EBEEF32
:101FA00010F061D90800F550DF6E1200200EE66EC9
:101FB000080E2EEF11F0D6EC16F0E552E552E55280
:101FC000F3CF14F0F4CF15F00001F31C1200146EDF
:101FD000156AD950010F4DD91450EE261550ED2237
:101FE0001200185E000E195AF70E18C0DBFFF80E2B
:101FF00019C0DBFF18C0E9FF19C0EAFF1200DBCFF0
:10200000F4FFF350F45C1200DB50E76E040EE7CFF0
:10201000DBFF12000A0EDBCF14F00B0EDBCF15F046
:102020000C0EDBCF16F00D0EDBCF17F01450151091
:10203000161017101200130EEECFDBFF140EEDCFAB
:10204000DBFF130EDBCF14F0140EDBCF15F0000115
:10205000800E15141200F70EDBCF18F0F80EDBCF50
:1020600019F01200050EDB50E66ED950130F01D99E
:10207000E552E750EE6EED6A12000A0EDBCF04F077
:102080000B0EDBCF05F00C0EDBCF06F00D0EDBCF19
:1020900007F01200DBCFE6FF150EDBCFE6FF050EE3
:1020A000DB50E552E724E552E7241200DB50CED89E
:1020B000010EF36E060EF3CFDBFF1200EE50EFCFF2
:1020C000EAFFE96E16C0EEFF17C0EEFF18C0EEFF84
:1020D0001200D9CFE6FFDACFE6FFE1CFD9FFE2CF9A
:1020E000DAFF1200DFCFE6FFE66A33EC18F0E552C4
:1020F000E552F3501200E76E080EE7CFDBFF120047
:10210000EECF14F0EECF15F0EFCF16F0176A1200F5
:10211000050EDBCF14F0150EDB50D88014541200DE
:10212000010EDBCF16F0020EDBCF17F0186A12009B
:10213000E552E5CFDAFFE7CFD9FF12000A0E14C04F
:10214000DBFF0B0E15C0DBFF1200D9500A0F39EF71
:1021500011F0F36E070EF3CFDBFF1200EECF14F099
:10216000EFCF15F01200010EDB2A020E1200FC0E5A
:10217000DBCFE6FFFD0EDBCFE6FF1200145E000EA4
:10218000155AF70E14C0DBFFF80E15C0DBFF14C0A4
:10219000E9FF15C0EAFF1200DA20EA6EEF2AEECF5F
:1021A000F6FF000EEF22EECFF7FFEF22EECFF8FFA3
:1021B0001200040EDBCFE6FF130EDB50E552E75CA6
:1021C0009ADFDB5004DF060EDB501200090EDB50F5
:1021D0000A0DF350DF24D00FE76E090EE7CFDBFFC7
:1021E000D1EF0FF0DB50F36E050EFFEF0FF0F70E9F
:1021F000DBCF14F0F80EDBCF15F01200DFCFE6FFD7
:10220000DBEF0FF028DF030EECDE80EF10F02DEC9B
:102210000BF0E552E552E552E55200091200BDDE31
:10222000EE50EFCFEAFFE96E010E1200130EDB5005
:10223000F36E040EFFEF0FF0040EDB50F36E090E89
:10224000FFEF0FF0DBCFE6FFDBEF0FF0E76E050EE1
:10225000E7CFDBFF12008BDFFEEF10F0DBCFE6FFF6
:1022600086DF07EF11F0D950F90FE96EFF0ECCEFC2
:1022700010F0E96E000EDA20EA6E12000F9E08D010
:102280000F9E07AE05D0066C071EE86A07220F8E68
:1022900007C001F006C000F0136A126A8E0E026ECB
:1022A000036A5CEF13F00D7E0F6A98EC13F0B0EC4C
:1022B00013F00FB640EF13F00FA20AD00FAA03D00D
:1022C0000FBE40EF13F00FA44CEF13F049EF13F0E3
:1022D0000FAA05D00FAC4CEF13F049EF13F00FA08D
:1022E0000AD00FA808D00FBE04D00FA402D055EF1B
:1022F00013F059EF13F0126A036A0D50085C116E67
:1023000010E305C013F006C000F007C001F008C0DC
:1023100010F00AC005F00BC006F00CC007F00F3A31
:1023200009D00AC013F00BC000F00CC001F00DC0C2
:1023300010F0116C0F9E0FBC0F8E10C002F00FB08A
:1023400088EF13F01A0E116088EF13F0026A086A22
:102350000FA408D0056C061E071E081EE86A062298
:10236000072208220FAC08D0136C001E011E021EAB
:10237000E86A002201220222046A115207E00834AE
:102380000732063205320432112EF9D705501326D2
:1023900006500022075001220850022204C012F009
:1023A0000F9E02AE0BD0126C131E001E011E021EE9
:1023B000E86A13220022012202220F8E02A006D018
:1023C000D8800132003213321232102A10C002F0CB
:1023D0005CEF13F00F6A98EC13F0B0EC13F00FB64B
:1023E00040EF13F00FA205D00FBA40EF13F047EF04
:1023F00013F00FBA53EF13F00FA005D00FB840EF52
:1024000013F053EF13F00FB847EF13F0036A7F0E8A
:102410000824026EE86A03220D50025EE86A035A3D
:102420001A0E106E086A126A136A006A016A0A506C
:10243000055E0B50065A0C50075A000E085A09E761
:102440000A5005260B5006220C500722000E0822C7
:1024500001D0128AD8900536063607360836D8904D
:102460001236133600360136102EE1D7075006100B
:102470000510D8A4128A5CEF13F00F6A98EC13F0E1
:10248000B0EC13F00FB640EF13F00FA205D00FB869
:1024900040EF13F047EF13F00FAA05D00FB040EF55
:1024A00013F047EF13F00FB002D00FA802D053EF94
:1024B00013F0036A0D500824026EE86A03227E0EB0
:1024C000025EE86A035A126A136A006A016A0C50D3
:1024D0000702F4CF01F0F3CF00F00B500702F350E6
:1024E0001326F4500022000E01220C500602F35075
:1024F0001326F4500022000E01220A500702F35066
:102500001226F4501322000E002201220B50060264
:10251000F3501226F4501322000E002201220C5018
:102520000502F3501226F4501322000E002201225D
:102530000A500602F4501226000E13220022012235
:102540000B500502F4501226000E13220022012225
:102550005CEF13F00F6A98EC13F00FB6B4EF12F0C3
:102560000FA20ED00FB405D07F0E076EFF0E066EC1
:102570001FD0800E076E066A1BD0076A066A18D045
:102580000FB0FBD78F0E0860EDD77E0E0864F5D72D
:102590008E0E085C05E0D89007320632082AF8D77C
:1025A0000FA406D0066C071EE86A072207AEE5D71F
:1025B0001200EBEC12F00FB6000C0FB0000C0FB4D1
:1025C000000C010CEBEC12F00FB6000C0FB0000C7D
:1025D0000FA4000C010C0F6A98EC13F0B0EC13F090
:1025E0000FB612000FAE08D00FA004D00FA802D073
:1025F0000F8012000F9012000D50085C0BE10C5080
:10260000075C08E10B50065C05E10A50055C02E13D
:102610000F801200D8A002D00F8E10D008500DC02D
:1026200008F00D6E07500CC007F00C6E06500BC082
:1026300006F00B6E05500AC005F00A6E0D50085CDE
:1026400010E0FF0F09E00F900FB403D00FAE0F841E
:1026500012000FAE0F9412000D2AD8900C320B32DC
:102660000A320A50055E0B50065A0C50075A07BE34
:10267000EAD7D890053606360736082EF8D7C8D7D9
:102680007F0E086EFF0E076E066E056E12007F0E3F
:102690000FBEFF0E086E02D07F0E086E800E076E12
:1026A000066A056AF3D70FAE04D0800E086E076A7B
:1026B000F7D7086A076AF4D70150001013101210F8
:1026C000F8E003BEF0D701BE0CD002500310EBE0DF
:1026D000D89012361336003601360206D8A003060B
:1026E000F2D70350D4E10228D2E012AE11D07F0E0F
:1026F000121402E113A00CD0132AE86A002201226E
:1027000007E3D880013200321332022A0228BFE0E8
:102710000250C9E013C005F000C006F00134076E96
:102720000230086E0732089E0FBE088E46EF13F087
:102730000736083602E30F840F7E06E10F80086A31
:10274000076A066A056A1200082803E0D880073283
:102750001200D890073202E10F8212000F86120099
:102760000C360D3602E30F8C0F7E06E10F880D6AE2
:102770000C6A0B6A0A6A12000D2803E0D8800C323A
:102780001200D8900C32EAE10F8A120007C013F051
:1027900006C012F006500B02F4CF05F0F3CF04F0A0
:1027A00007500C02F4CF07F0F3CF06F00B02F35002
:1027B0000526F4500622E86A072212500C02F35054
:1027C0000526F4500622E86A07220CAEECEF13F05F
:1027D0001250065E1350075A13AE000C0B50065EE3
:1027E0000C50075A000CD9CFE6FFDACFE6FFFA0EFD
:1027F000E3CFD9FFFB0EE3CFDAFFFD0EE35209E78B
:102800002D0EDE6EFC0EE31EE32AFD0ED8B4E306A9
:10281000E31EE652E652E652FD0EE124E76EFF0E9D
:10282000E220E46EE652F70EE3CFE6FFF70EE3CFC9
:10283000E6FF63EC14F0F90EE124E96EFF0EE220EE
:10284000EA6E53EC14F00AE150EC14F009E153EC99
:1028500014F008E150EC14F007E108D05EEC14F03D
:1028600059EC14F05EEC14F059EC14F05EEC14F03A
:10287000DE6AF90EE126FF0EE222FF0EE3CFDAFF59
:10288000E552FF0EE3CFD9FFE552FC0EE124E96EDD
:10289000FF0EE220EA6EEECFF3FFEFCFF4FF12005F
:1028A000EF380F0B1200EF500F0B02E1EE52D884FD
:1028B0001200EF380F0B300FDE6E1200EE500F0BD0
:1028C000300FDE6E1200FC0EE3CFE9FFFD0EE3CF0A
:1028D000EAFF100EE66EEE6AEE6AEF6AD890FD0E21
:1028E000E336FE0EE336ED36ED36EF36FF0EE30649
:1028F00009E084EC14F0EE5284EC14F0EE5284EC17
:1029000014F0EDD7E56E1200030EEF24E8B6EF6E7B
:10291000300EEF24E8BEEF6E000CD9CFE6FFDACF21
:10292000E6FFF80EE3CFD9FFF90EE3CFDAFFE65268
:10293000E652E652E652E652FB0EE124E76EFF0E47
:10294000E220E46EE652F30EE3CFE6FFF30EE3CFB0
:10295000E6FFF30EE3CFE6FFF30EE3CFE6FF12EC64
:1029600015F0F50EE124E96EFF0EE220EA6EFFECB1
:1029700014F019E102EC15F018E1FFEC14F017E186
:1029800002EC15F016E1FFEC14F015E102EC15F085
:1029900014E1FFEC14F013E102EC15F012E1FFEC8E
:1029A00014F011E112D008EC15F00DEC15F008EC64
:1029B00015F00DEC15F008EC15F00DEC15F008EC29
:1029C00015F00DEC15F008EC15F00DEC15F0DE6AC5
:1029D000F50EE126FF0EE222FF0EE3CFDAFFE5520D
:1029E000FF0EE3CFD9FFE552FA0EE124E96EFF0EA8
:1029F000E220EA6EEECFF3FFEFCFF4FF1200EF38E4
:102A00000F0B1200EF500F0B02E1EE52D8841200B0
:102A1000EF380F0B300FDE6E1200EE500F0B300F41
:102A2000DE6E1200FA0EE3CFE9FFFB0EE3CFEAFF02
:102A3000200EE66EEE6AEE6AEE6AEE6AEF6AD890F3
:102A4000FB0EE336FC0EE336FD0EE336FE0EE336F8
:102A5000ED36ED36ED36ED36EF36FF0EE3060FE0E0
:102A600041EC15F0EE5241EC15F0EE5241EC15F050
:102A7000EE5241EC15F0EE5241EC15F0E1D7E56E67
:102A80001200030EEF24E8B6EF6E300EEF24E8BE1E
:102A9000EF6E000CD9CFE6FFE1CFD9FF020EE126A1
:102AA000FD0EDBCFDEFFDBCFDDFFD9CFE9FFDACFD5
:102AB000EAFFEE06000EED5AEECF14F0EDCF15F062
:102AC0001450151001E0F1D7020EE15C02E2E16A58
:102AD000E552E16EE552E7CFD9FF1200D9CFE6FF0C
:102AE000E1CFD9FFF29A010ED56EFC0ED76E190E0A
:102AF000D66ED950FD0FE96EFF0EDA20EA6E000E99
:102B0000D880EE54000EED540EE2D58EF2A4FED71E
:102B1000F294FD0EDB06FE0E01E2DB06FC0ED76E24
:102B2000190ED66EE6D7D56AE552E7CFD9FF120067
:102B3000F29A070ED56EC20ED76EF70ED66ED58EF0
:102B4000F2A4FED7F294D56AC20ED76EF70ED66EF7
:102B500012000E0EF66E000EF76E000EF86E0001FB
:102B60000900F550D36F0900F550D46F03E1D36726
:102B700001D03DD00900F550CE6F0900F550CF6F60
:102B80000900F550D06F09000900F550E96E090001
:102B9000F550EA6E090009000900F550D16F0900EF
:102BA000F550D26F09000900F6CFD5F0F7CFD6F077
:102BB000F8CFD7F0CEC0F6FFCFC0F7FFD0C0F8FFF8
:102BC0000001D15302E1D25307E00900F550EE6E47
:102BD000D107F8E2D207F9D7D5C0F6FFD6C0F7FF84
:102BE000D7C0F8FF0001D307000ED45BBFD7120097
:102BF000D9CFE6FFDACFE6FFE1CFD9FFE2CFDAFFA8
:102C0000E652E652E652E652D950F90F146EFF0E24
:102C1000DA20156E14C0DEFFDD6EDECFE6FFDDCFFD
:102C2000E6FFF90EDBCFE6FFFA0EDBCFE6FFFB0E89
:102C3000DBCFE6FFFC0EDBCFE6FFFD0EDBCFE6FFD2
:102C400043EC0BF0146E070EE15C02E2E16AE55220
:102C5000E16E1450020EF3CFDBFF030EF4CFDBFF67
:102C6000020EDBCF14F0030EDBCF15F014C0F3FF20
:102C700015C0F4FF040EE15C02E2E16AE552E16E88
:102C8000E552E5CFDAFFE7CFD9FF1200FB0EE3CF25
:102C9000F6FFFC0EE3CFF7FFFD0EE3CFF8FFFE0ECD
:102CA000E3CFE9FFFF0EE3CFEAFFE9CFF3FFEACF7F
:102CB000F4FF0900F5CFEFFFEE66FBD71200FE0E22
:102CC000E3CFE9FFFF0EE3CFEAFFF36AF46AEE52C7
:102CD00003E0F34AF42AFBD71200FF0EE3CFF8FF1C
:102CE000E552FF0EE3CFF7FFE552FF0EE3CFF6FF0D
:102CF000E552E66AE66AE66A0900F55209E0FD0E69
:102D0000E32A05E1FE0EE32A02E1FF0EE32AF4D7EF
:102D1000FD0EE3CF05F0FE0EE3CF06F0FF0EE3CF8E
:102D200007F0120053756D31363D20253035642093
:102D3000736F697420257320B043004D53502043B6
:102D40004831202530356420736F69742025732045
:102D5000566F6C7473202563004C656374204D536B
:102D6000502043483020783130202530356420739E
:102D70006F69742054656D703D25732054456D70E6
:102D800020B04320256300416C696D206475204D9F
:102D90006F6E74616765203D352E30202D3E2025F5
:102DA0007325630025732563007800FFD9CFE6FF04
:102DB000DACFE6FFE1CFD9FFE2CFDAFFFB0EDBCFC0
:102DC00014F0FC0EDBCF15F00001800E15141AE193
:102DD000FB0EDBCFE9FFFC0EDBCFEAFFEECFF3FF0C
:102DE000EDCFF4FFEE2A000EEF22F3CFE9FFF4CF90
:102DF000EAFFFD0EDBCFEFFFEF50156AF36E15C053
:102E0000F4FF10D0FB0EDB50FE0806E1FD0EDBCF19
:102E1000E6FF63EC18F005D0FD0EDBCFE6FF03EC18
:102E200000F0E552E552E5CFDAFFE7CFD9FF120017
:102E3000D9CFE6FFDACFE6FFE1CFD9FFE2CFDAFF65
:102E4000AC6AAB6AFD0EDBB0AC88DBA202D0AC8C06
:102E5000AB8CDBB4AC8EDBA602D0AB8801D0AB8AE6
:102E6000DBB8AC84DBBAAB86DBAC02D09D8A01D088
:102E70009D9ADBAE02D09D8801D09D98FB0EDB5061
:102E8000AF6EFC0EDBCF15F015C014F0156A1450B0
:102E9000B06EAC8AAB8EE552E5CFDAFFE7CFD9FF53
:102EA000120004500902F3CF00F0F4CF01F00A023F
:102EB000F3500126000EF420026E04500B02F35072
:102EC0000226000EF420036E04500C02F350032679
:102ED00005500902F3500126F4500222000E03228D
:102EE00005500A02F3500226F450032205500B024B
:102EF000F350032606500902F3500226F450032231
:102F000006500A02F350032607500902F350032625
:102F100012002E2E2E004F7363696C6C20696E7444
:102F200065726E652031364D687A200D0A00433196
:102F3000383A2031384632364B32325F546573743A
:102F40005F4D4350365332365F4C4D3335445A5FF4
:102F50003134303132342E63200D0A004C4D33357C
:102F6000445A2020306D5620402030B043200D0AB6
:102F700000200D0A00200D0A00FF036A026A016AA0
:102F8000006A200EE76ED8900436053606360736FE
:102F900000360136023603360950005C0A500158EB
:102FA0000B5002580C50035809E30950005E0A50B8
:102FB000015A0B50025A0C50035A042AE72EE4D748
:102FC0001200D9CFE6FFDACFE6FFE1CFD9FFE2CF9B
:102FD000DAFFE652F20E0101F917ABAC03D0F9911A
:102FE000ABB0F981ABB4F985ABB2F987AE50DF6E07
:102FF000DF50E552E552E5CFDAFFE7CFD9FF120007
:10300000D9CFE6FFDACFE6FFE1CFD9FFE2CFDAFF93
:10301000E652E652FC0EDBCFDEFFDBCFDDFF010E1A
:10302000DB50CF6EDF50CE6EE552E552E552E5CF74
:10303000DAFFE7CFD9FF1200D9CFE6FFDACFE6FFFC
:10304000E1CFD9FFE2CFDAFFACAC04D0AC90010104
:10305000F9B3AC80FD0EDB50AD6EE552E5CFDAFF83
:10306000E7CFD9FF1200F36AF46AFF0EE124E96E9C
:10307000FF0EE220EA6EED6607D02F0EEF6404D05B
:103080003A0EEF6001D0F32A1200380EF36E00EE14
:1030900000F00F0E01D81200EA6002D0EE6AFCD7F1
:1030A000F350E9601200EE6AFCD71EEE00F02EEE3F
:1030B00000F0F86A0F9CA9EC15F08AEC18F05EECB1
:1030C00008F0FBD71200FF0EE350ACBA04D0AF6A91
:1030D000AB8EAC8A949CACA2FED7AD6EF36EF46A54
:1030E0001200C450176E166AC3501610F36E17C044
:1030F000F4FF1200303132333435363738396162FB
:103100006364656600FFC250020B01E0010E12000D
:10311000C28212001200122F162F2E2F5C2F712F39
:10312000752F31384632364B3232204D43503653AC
:10313000323620414F500000000000000000000027
:10314000000000000000000000000000000000007F
:10315000000000000000000000000000000000006F
:10316000000000000000000000000000000000005F
:103170000000313233343536373839303132333478
:1031800035360000FFFFFFFFFFFFFFFFFFFFFFFFE0
:10319000FFFFFFFFFFFFFFFFFFFFFFFFFFFFFFFF3F
:1031A000FFFFFFFFFFFFFFFFFFFFFFFFFFFFFFFF2F
:1031B000FFFFFFFFFFFFFFFFFFFFFFFFFFFFFFFF1F
:1031C000FFFFFFFFFFFFFFFFFFFFFFFFFFFFFFFF0F
:0200000400F00A
:1000000031384632364B32325F74657374735F64D5
:1000100069766572732E6D637020202020200D009C
:10002000496E697420506F725420436F6D20525393
:100030003233322031393230306264732E200D0079
:100040002E2E2E2E2E2E2E2E2E2E2E2E2E2E2E2ED0
:1000500020203C4553433E206578697420200D00E4
:1000600041766563205541525420484152445741DE
:1000700052452E2E2E2E2E2E2E2E2E2E2E200D00C2
:100080002020202020202020202020202020202070
:1000900020202020202020202020202020200D0093
:1000A0007061756C666A756A6F40667265652E660A
:1000B000722032332F30312F32303134200D000096
:1000C0004D504C4142204944452056382E3930206D
:1000D000204331382076332E34352E30310D000058
:1000E0002020202020202020202020202020202010
:1000F000202020202020202020200D0A00000000A9
:10010000FFFFFFFFFFFFFFFFFFFFFFFFFFFFFFFFFF
:10011000FFFFFFFFFFFFFFFFFFFFFFFFFFFFFFFFEF
:10012000FFFFFFFFFFFFFFFFFFFFFFFFFFFFFFFFDF
:10013000FFFFFFFFFFFFFFFFFFFFFFFFFFFFFFFFCF
:10014000FFFFFFFFFFFFFFFFFFFFFFFFFFFFFFFFBF
:10015000FFFFFFFFFFFFFFFFFFFFFFFFFFFFFFFFAF
:10016000FFFFFFFFFFFFFFFFFFFFFFFFFFFFFFFF9F
:10017000FFFFFFFFFFFFFFFFFFFFFFFFFFFFFFFF8F
:10018000FFFFFFFFFFFFFFFFFFFFFFFFFFFFFFFF7F
:10019000FFFFFFFFFFFFFFFFFFFFFFFFFFFFFFFF6F
:1001A000FFFFFFFFFFFFFFFFFFFFFFFFFFFFFFFF5F
:1001B000FFFFFFFFFFFFFFFFFFFFFFFFFFFFFFFF4F
:1001C000FFFFFFFFFFFFFFFFFFFFFFFFFFFFFFFF3F
:1001D000FFFFFFFFFFFFFFFFFFFFFFFFFFFFFFFF2F
:1001E000FFFFFFFFFFFFFFFFFFFFFFFFFFFFFFFF1F
:1001F000FFFFFFFFFFFFFFFFFFFFFFFFFFFFFFFF0F
:1002000054657374204D43503653323620202020DD
:100210002020000031384632364B3232204331380C
:100220002031364D487A0000FFFFFFFFFFFFFFFF40
:10023000FFFFFFFFFFFFFFFFFFFFFFFFFFFFFFFFCE
:10024000FFFFFFFFFFFFFFFFFFFFFFFFFFFFFFFFBE
:10025000FFFFFFFFFFFFFFFFFFFFFFFFFFFFFFFFAE
:10026000FFFFFFFFFFFFFFFFFFFFFFFFFFFFFFFF9E
:10027000FFFFFFFFFFFFFFFFFFFFFFFFFFFFFFFF8E
:10028000FFFFFFFFFFFFFFFFFFFFFFFFFFFFFFFF7E
:10029000FFFFFFFFFFFFFFFFFFFFFFFFFFFFFFFF6E
:1002A000FFFFFFFFFFFFFFFFFFFFFFFFFFFFFFFF5E
:1002B000FFFFFFFFFFFFFFFFFFFFFFFFFFFFFFFF4E
:1002C000FFFFFFFFFFFFFFFFFFFFFFFFFFFFFFFF3E
:1002D000FFFFFFFFFFFFFFFFFFFFFFFFFFFFFFFF2E
:1002E000FFFFFFFFFFFFFFFFFFFFFFFFFFFFFFFF1E
:1002F000FFFFFFFFFFFFFFFFFFFFFFFFFFFFFFFF0E
:10030000FFFFFFFFFFFFFFFFFFFFFFFFFFFFFFFFFD
:10031000FFFFFFFFFFFFFFFFFFFFFFFFFFFFFFFFED
:10032000FFFFFFFFFFFFFFFFFFFFFFFFFFFFFFFFDD
:10033000FFFFFFFFFFFFFFFFFFFFFFFFFFFFFFFFCD
:10034000FFFFFFFFFFFFFFFFFFFFFFFFFFFFFFFFBD
:10035000FFFFFFFFFFFFFFFFFFFFFFFFFFFFFFFFAD
:10036000FFFFFFFFFFFFFFFFFFFFFFFFFFFFFFFF9D
:10037000FFFFFFFFFFFFFFFFFFFFFFFFFFFFFFFF8D
:10038000FFFFFFFFFFFFFFFFFFFFFFFFFFFFFFFF7D
:10039000FFFFFFFFFFFFFFFFFFFFFFFFFFFFFFFF6D
:1003A000FFFFFFFFFFFFFFFFFFFFFFFFFFFFFFFF5D
:1003B000FFFFFFFFFFFFFFFFFFFFFFFFFFFFFFFF4D
:1003C000FFFFFFFFFFFFFFFFFFFFFFFFFFFFFFFF3D
:1003D000FFFFFFFFFFFFFFFFFFFFFFFFFFFFFFFF2D
:1003E000FFFFFFFFFFFFFFFFFFFFFFFFFFFFFFFF1D
:1003F000FFFFFFFFFFFFFFFFFFFFFFFFFFFFFFFF0D
:020000040030CA
:0E0000000028193C009D84000FC00FE00F4047
:020000040020DA
:08000000FFFFFFFFFFFFFFFF00
:00000001FF
